BL51 BANKED LINKER/LOCATER V5.03                                                        04/30/2012  12:50:05  PAGE 1


BL51 BANKED LINKER/LOCATER V5.03, INVOKED BY:
D:\KEIL\C51\BIN\BL51.EXE Text1.obj TO 双机通信


MEMORY MODEL: SMALL


INPUT MODULES INCLUDED:
  Text1.obj (TEXT1)
  D:\KEIL\C51\LIB\C51S.LIB (?C_STARTUP)
  D:\KEIL\C51\LIB\C51S.LIB (?C_INIT)


LINK MAP OF MODULE:  双机通信 (TEXT1)


            TYPE    BASE      LENGTH    RELOCATION   SEGMENT NAME
            -----------------------------------------------------

            * * * * * * *   D A T A   M E M O R Y   * * * * * * *
            REG     0000H     0008H     ABSOLUTE     "REG BANK 0"
            DATA    0008H     000EH     UNIT         ?DT?TEXT1
            DATA    0016H     0004H     UNIT         _DATA_GROUP_
            IDATA   001AH     0001H     UNIT         ?STACK

            * * * * * * *   C O D E   M E M O R Y   * * * * * * *
            CODE    0000H     0003H     ABSOLUTE     
                    0003H     0020H                  *** GAP ***
            CODE    0023H     0003H     ABSOLUTE     
                    0026H     07DAH                  *** GAP ***
            CODE    0800H     008CH     UNIT         ?C_C51STARTUP
            CODE    088CH     0055H     UNIT         ?PR?MAIN?TEXT1
            CODE    08E1H     001FH     UNIT         ?PR?_DELAY?TEXT1
            CODE    0900H     001AH     UNIT         ?PR?SERIAL_INIT?TEXT1
            CODE    091AH     000DH     UNIT         ?PR?SERIAL_INTE?TEXT1
            CODE    0927H     000DH     UNIT         ?C_INITSEG



OVERLAY MAP OF MODULE:   双机通信 (TEXT1)


SEGMENT                          DATA_GROUP 
  +--> CALLED SEGMENT          START    LENGTH
----------------------------------------------
?C_C51STARTUP                  -----    -----
  +--> ?PR?MAIN?TEXT1
  +--> ?C_INITSEG

?PR?MAIN?TEXT1                 0016H    0004H
  +--> ?PR?SERIAL_INIT?TEXT1
  +--> ?PR?_DELAY?TEXT1



SYMBOL TABLE OF MODULE:  双机通信 (TEXT1)

  VALUE           TYPE          NAME
BL51 BANKED LINKER/LOCATER V5.03                                                      04/30/2012  12:50:05  PAGE 2


  ----------------------------------

  -------         MODULE        TEXT1
  C:0000H         SYMBOL        _ICE_DUMMY_
  D:0090H         PUBLIC        P1
  D:00A0H         PUBLIC        P2
  B:00A8H.7       PUBLIC        EA
  C:091AH         PUBLIC        serial_inte
  B:00A8H.4       PUBLIC        ES
  C:0900H         PUBLIC        serial_init
  B:0098H.0       PUBLIC        RI
  B:0098H.1       PUBLIC        TI
  C:088CH         PUBLIC        main
  D:0099H         PUBLIC        SBUF
  D:0087H         PUBLIC        PCON
  D:0098H         PUBLIC        SCON
  D:0089H         PUBLIC        TMOD
  D:0008H         PUBLIC        dat
  D:008DH         PUBLIC        TH1
  D:008BH         PUBLIC        TL1
  B:00A0H.1       PUBLIC        p21
  B:0088H.6       PUBLIC        TR1
  D:0012H         PUBLIC        f
  D:0014H         PUBLIC        j
  C:08E1H         PUBLIC        _delay
  -------         PROC          _DELAY
  D:0006H         SYMBOL        x
  -------         DO            
  D:0004H         SYMBOL        k
  -------         ENDDO         
  C:08E1H         LINE#         8
  C:08E1H         LINE#         9
  C:08E1H         LINE#         11
  C:08EBH         LINE#         12
  C:08EBH         LINE#         13
  C:08FFH         LINE#         14
  C:08FFH         LINE#         15
  -------         ENDPROC       _DELAY
  -------         PROC          SERIAL_INIT
  C:0900H         LINE#         17
  C:0900H         LINE#         18
  C:0900H         LINE#         19
  C:0903H         LINE#         20
  C:0905H         LINE#         21
  C:0908H         LINE#         22
  C:090AH         LINE#         23
  C:090DH         LINE#         24
  C:0910H         LINE#         25
  C:0913H         LINE#         26
  C:0915H         LINE#         27
  C:0917H         LINE#         28
  C:0919H         LINE#         29
  -------         ENDPROC       SERIAL_INIT
  -------         PROC          SERIAL_INTE
  C:091AH         LINE#         31
  C:091AH         LINE#         33
  C:091CH         LINE#         34
BL51 BANKED LINKER/LOCATER V5.03                                                      04/30/2012  12:50:05  PAGE 3


  C:091FH         LINE#         35
  C:091FH         LINE#         36
  C:0921H         LINE#         37
  C:0924H         LINE#         44
  C:0924H         LINE#         45
  C:0926H         LINE#         46
  -------         ENDPROC       SERIAL_INTE
  -------         PROC          MAIN
  -------         DO            
  D:0016H         SYMBOL        i
  D:0018H         SYMBOL        t
  -------         ENDDO         
  C:088CH         LINE#         48
  C:088CH         LINE#         49
  C:088CH         LINE#         51
  C:088FH         LINE#         52
  C:0892H         LINE#         53
  C:0892H         LINE#         54
  C:0892H         LINE#         55
  C:08A2H         LINE#         56
  C:08A2H         LINE#         57
  C:08ABH         LINE#         58
  C:08B2H         LINE#         59
  C:08C0H         LINE#         60
  C:08C0H         LINE#         61
  C:08C3H         LINE#         62
  C:08CBH         LINE#         63
  C:08CEH         LINE#         64
  C:08D0H         LINE#         65
  C:08D8H         LINE#         66
  C:08DFH         LINE#         67
  C:08DFH         LINE#         68
  -------         ENDPROC       MAIN
  -------         ENDMOD        TEXT1

******************************************************************************
* RESTRICTED VERSION WITH 0800H BYTE CODE SIZE LIMIT; USED: 00B1H BYTE ( 8%) *
******************************************************************************

Program Size: data=27.0 xdata=0 code=314
LINK/LOCATE RUN COMPLETE.  0 WARNING(S),  0 ERROR(S)
